:10000000FF28000000000000B22A8207A0349034CC
:100010005034603482070C340934033406348207C8
:10002000103420341C341C341C341C34003414347C
:100030002A342B342A342B342A342B342A342B34CC
:1000400021340234033404340534063407340834CC
:1000500024341A34253425342434243425340D34FE
:1000600028342934283429342834293428342934AC
:1000700024341734243416342534153425341434F8
:100080002434133412341134253410340F340E3424
:100090002A3420342B3420342A3420342B341534A1
:1000A0002734203426342034273420342634233493
:1000B00021341934213421342134213421342134A0
:1000C00026340234273403342634043427340534E8
:1000D00026340634273407342634083427341234BF
:1000E00021341D341D341D341D3421342134003499
:1000F0001334263427342634273416342634273450
:100100000934293427342534233421340234033488
:100110000434053406340734083409340A341534F9
:100120002A342B342A342B342A342B342A342B34DB
:100130002134143413341234113410340E34023494
:10014000263426342734173426342634273405340D
:1001500026342634273417342634263427341A34E8
:1001600028342934283429342834293428342934AB
:100170002434073424340234253408342534033439
:10018000243407342434153425340534253401341B
:10019000293420342A342034293420342A34203499
:1001A000273426342734263427342634273426347B
:1001B0001A34213421340134053408341134143410
:1001C00026340334273405342634043427340634E3
:1001D00026340734273416342634173482077F3404
:1001E0007F34483448343C343C34323432342A345A
:1001F0002A3423342334FF34FF347F347F3483168E
:100200000D308600103085006400033081008312B9
:10021000850186010C3084008001840A04084E3C6C
:10022000031D0C29422290308B002D309200393072
:10023000A4000D1A52298D1C26292208283C0319D6
:1002400025292208013C031D26290D152022DD2128
:10025000F821702264003208FB3C0319452932085A
:10026000FC3C03193729861D4829061D4529FF3006
:100270001C02031C19299D0A37301D02031C192971
:100280009C019D010C14582119292F228A22192919
:100290000C1F19292D08AE00E4220C132D08900024
:1002A0006B211929FE30AE00E422FF280D1608004C
:1002B000910A11081108DC3C0318652900309100EF
:1002C000B10A3108033C0319562911080F20AE006A
:1002D000E4222E0890001008003C03199C29100805
:1002E000203C0319A2291008213C0319A529100854
:1002F000173C0318B6291008193C0319BD2910082A
:100300001A3C0319C22910081B3C0319C7291008FD
:100310001C3C0319CA2910081D3C0319CD291008DB
:100320001E3C0319D02910081F3C0319D3291008BB
:100330002B3C0318A92908008D103930A400003087
:10034000A0000D158C100C1008008C148C160C14C9
:1003500008008C120C1410080F39EE2092008C1437
:10036000101CB4290C1508000C1108001008A0007E
:100370000D153930A4008D1008003C30A400173052
:100380008E00DA295030A4000A308E00DA290630B7
:10039000AF00D6290C30AF00D6291830AF00D629CF
:1003A0002D30AF00D6294630AF00D62900308E0060
:1003B0003930A4000D158D1408008D1DF7298D1CF2
:1003C000EB292208083C0319E8290130A000ED2997
:1003D0000E08A000ED290D1DF7290D118D111F30FC
:1003E0002005AB000310AB0DAB0D2B0DA1000800D9
:1003F00024082302031C0800A3013008003C031951
:10040000032AB0030800220821020319112A031C41
:100410000B2AA20A0C2AA203033022050A20850017
:1004200008000D1D1C2A8D158D1C1C2A2208003C5D
:10043000031D1D2A2F08B00008000430B00008007A
:10044000811D08008101940A930A980A9A0A9C0A5D
:10045000A30A0800811F08008101A30A08000C1AE2
:100460003E2AFF301A02031C3D2A9B0A1A301B0247
:10047000031C3D2A9A019B010C160800051E3D2A0B
:100480000C125829BE30A2000030A100B430A400E4
:1004900064002022F8212208003C0319502A482A2F
:1004A000B430A4001430A20064002A22F8212208EB
:1004B000003C03195C2A542A3930A4001430A100EE
:1004C00064002022F8212208083C0319682A602AC7
:1004D00064000130A0000830A2000830A10008002C
:1004E0000C1C08008C1C08008C1A022B1208140229
:1004F000031C080094010C1D7F2A950A802A95038D
:10050000033015050520F039AA0006080F392A0422
:1005100086000800051E9A2A0D18942A0130AE00A4
:10052000E4220130A0000D150C14980199019E01E0
:100530000D140800FF301802031CB12A990A5A3022
:100540001902031CB12A99010C100D1CB12A20308C
:10055000AE00E4229E0A1C301E02031CB12A0D10BC
:100560000D160800A900030E8312A8000618DA2A47
:10057000FD220618DA2AFB220830A600060CA70C7A
:10058000FB22A603031DBE2A061CDA2A2708AD009B
:100590000C172D08FB3C0319E12A2D08FD3C03191B
:1005A000E12A2D08FC3C0319E12A2D08FE3C031D1D
:1005B000DA2A0D1664008B10280E8300A90E290E6E
:1005C00009002D08B200DA2A86142E08AC00FB229E
:1005D0000830AB00AC0C0318EF2A8614F02A861002
:1005E000FB22AB03031DEA2A861064008101F92275
:1005F00008006430FE2A1D30FE2A0F30AA00AA0B24
:10060000FF2A080002301302031C112B93018F03F1
:1006100003190E2B8F0303190E2B112B960A03308F
:1006200096050130160203192D2B0230160203190C
:100630003D2B0330160203194D2B103097070F087E
:1006400017020318282B06080F39A0388600080067
:1006500006080F39903886000800103097070F08F9
:1006600017020318382B06080F3990388600080047
:1006700006080F39503886000800103097070F0819
:1006800017020318482B06080F3950388600080057
:1006900006080F39603886000800103097070F08E9
:1006A00017020318582B06080F3960388600080017
:0A06B00006080F39A0388600080084
:02400E00F53F7C
:00000001FF
